:020000040000FA
:100000000A02040000000000D80A0000D80A00001C
:10001000D80A0000D80A0000D80A0000D80A000058
:10002000D80A0000D80A0000D80A0000D80A000048
:10003000D80A0000D80A0000D80A0000D80A000038
:10004000D80A0000E0070000D80A0000D80A000023
:10005000D80A0000D80A0000D80A0000D80A000018
:10006000D80A0000D80A0000D80A0000D80A000008
:10007000D80A0000D80A0000D80A0000D80A0000F8
:10008000D80A0000D80A0000D80A0000D80A0000E8
:10009000D80A0000D80A0000D80A0000D80A0000D8
:1000A000D80A0000D80A0000D80A0000D80A0000C8
:1000B000D80A0000D80A0000D80A0000D80A0000B8
:1000C000D80A0000D80A0000D80A0000D80A0000A8
:1000D000D80A0000D80A0000D80A0000D80A000098
:1000E000D80A0000D80A0000D80A0000D80A000088
:1000F000D80A0000D80A0000D80A0000D80A000078
:10010000D80A0000D80A0000D80A0000D80A000067
:10011000D80A0000D80A0000D80A0000D80A000057
:10012000D80A0000D80A0000D80A0000D80A000047
:10013000D80A0000D80A0000D80A0000D80A000037
:10014000D80A0000D80A0000D80A0000D80A000027
:10015000D80A0000D80A0000D80A0000D80A000017
:10016000D80A0000D80A0000D80A0000D80A000007
:10017000D80A0000D80A0000D80A0000D80A0000F7
:10018000D80A0000D80A0000D80A0000D80A0000E7
:10019000D80A0000D80A0000D80A0000D80A0000D7
:1001A000D80A0000D80A0000D80A0000D80A0000C7
:1001B000D80A0000D80A0000D80A0000D80A0000B7
:1001C000D80A0000D80A0000D80A0000D80A0000A7
:1001D000D80A0000D80A0000D80A0000D80A000097
:1001E000D80A0000D80A0000D80A0000D80A000087
:1001F000D80A0000D80A0000D80A0000D80A000077
:10020000FFFFFF00FFFFFF00D80A0000D80A000030
:10021000D80A0000D80A0000D80A0000D80A000056
:10022000D80A0000D80A0000D80A0000D80A000046
:10023000D80A0000D80A0000D80A0000D80A000036
:10024000D80A0000E0070000D80A0000D80A000021
:10025000D80A0000D80A0000D80A0000D80A000016
:10026000D80A0000D80A0000D80A0000D80A000006
:10027000D80A0000D80A0000D80A0000D80A0000F6
:10028000D80A0000D80A0000D80A0000D80A0000E6
:10029000D80A0000D80A0000D80A0000D80A0000D6
:1002A000D80A0000D80A0000D80A0000D80A0000C6
:1002B000D80A0000D80A0000D80A0000D80A0000B6
:1002C000D80A0000D80A0000D80A0000D80A0000A6
:1002D000D80A0000D80A0000D80A0000D80A000096
:1002E000D80A0000D80A0000D80A0000D80A000086
:1002F000D80A0000D80A0000D80A0000D80A000076
:10030000D80A0000D80A0000D80A0000D80A000065
:10031000D80A0000D80A0000D80A0000D80A000055
:10032000D80A0000D80A0000D80A0000D80A000045
:10033000D80A0000D80A0000D80A0000D80A000035
:10034000D80A0000D80A0000D80A0000D80A000025
:10035000D80A0000D80A0000D80A0000D80A000015
:10036000D80A0000D80A0000D80A0000D80A000005
:10037000D80A0000D80A0000D80A0000D80A0000F5
:10038000D80A0000D80A0000D80A0000D80A0000E5
:10039000D80A0000D80A0000D80A0000D80A0000D5
:1003A000D80A0000D80A0000D80A0000D80A0000C5
:1003B000D80A0000D80A0000D80A0000D80A0000B5
:1003C000D80A0000D80A0000D80A0000D80A0000A5
:1003D000D80A0000D80A0000D80A0000D80A000095
:1003E000D80A0000D80A0000D80A0000D80A000085
:1003F000D80A0000D80A0000D80A0000D80A000075
:1004000004020000001A000018120000100E000084
:10041000080000004507A90000002000403A8800BD
:100420002F97200000DF200000018800000000005E
:1004300081E0A80000002000A00188004440A8003E
:100440002CA3EF00C001200020168800000020002F
:1004500060168800C022EF00C822EF00C0A2A800EA
:10046000C022A800C002A800C9E2A800C9C2A80012
:100470006860A8006840A8006960A8006980A800BA
:100480000000EB00100009000060FE000000E90021
:10049000FCFF3A004027AE00050037004027A900C6
:1004A0000028EC00A00020000008E30037013D0018
:1004B000CE0A020000000000104088000060FE002C
:1004C00040802000DC02FC00B60009000018EB00B0
:1004D000F0FF270040418800600020000208E30090
:1004E000010039000228EF00104080000060010088
:1004F000050037002200370039003700630037005D
:1005000081003700D00037000000200060418800E3
:100510005007200080428800A00E2000A0438800E1
:10052000A0F32B00A0418800F0FF2B00C042880000
:10053000600C2C00E04388001000200080418800FF
:10054000A0428800C043880090418800B0428800E3
:10055000D0438800C001200070418800904288008C
:10056000B0438800808920001A00090030E0A00014
:1005700099C8A900ABC8A900BDC8A90016013700D9
:10058000E0282800A0418800E0512800C0428800EF
:10059000D07A2800E04388001000200080418800C5
:1005A000A0428800C043880090418800B042880083
:1005B000D04388008003200070418800904288006A
:1005C000B0438800808920001A00090030E0A000B4
:1005D00099C8A900B1C8A900C9C8A900FE00370080
:1005E00000002000604188007023200080428800C5
:1005F000E0462000A0438800A0CE2500A04188004E
:10060000F0FF2500C0428800701C2600E0438800EF
:100610001000200080418800A0428800C04388006C
:1006200090418800B0428800D043880040002000FC
:100630007041880050002000904288006000200037
:10064000B0438800808920001A00090030E0A00033
:1006500099C8A900ABC8A900BDC8A9003C28A8003A
:100660006028A8008428A80010002000C04188004D
:10067000E04288000044880010002000D04188003B
:10068000F042880010448800D300370000002000AA
:10069000604188005007200080428800A00E2000A2
:1006A000A0438800A0F32B00A0418800F0FF2B009E
:1006B000C0428800600C2C00E0438800100020003D
:1006C00080418800A0428800C04388009041880093
:1006D000B0428800D0438800C001200070418800EB
:1006E00090428800B0438800808920001A000900E9
:1006F00030E0A00099C8A900ABC8A900CDC8A900E6
:100700008408A800B40037000468A8000000200096
:100710006041880080428800A043880030FF2100AB
:10072000A0418800F0FF2F00C0428800F0FF2F009A
:10073000E04388001000200080418800F00F200076
:10074000A042880010002000C0438800F00F200065
:100750009041880000002000B0428800D04388000B
:100760005000200070418800000020009042880066
:10077000C0012000B0438800E08C20001A0009006E
:1007800030E0A000CFC8A900E1C8A900F3C8A900C3
:10079000910037000001200060418800F0FF2F0029
:1007A000A04188001000200080418800904188000E
:1007B000D001200070418800808920001A000900C3
:1007C00030E0A00099C8A9003C28A80082003700AA
:1007D0000001200080428800F0FF2F00C042880006
:1007E00010002000A0428800B0428800D001200004
:1007F00090428800808920001A00090030E0A000A3
:10080000ABC8A9006028A8007300370000012000D1
:10081000A0438800F0FF2F00E04388001000200074
:10082000C0438800D0438800D0012000B043880036
:10083000808920001A00090030E0A000BDC8A9008E
:100840008428A80064003700000020006041880070
:10085000002020008042880000402000A043880043
:10086000F0FF2F00A0418800C0428800E0438800CC
:100870001000200080418800A0428800C04388000A
:1008800090418800B0428800D0438800C001200019
:100890007041880090428800B04388008089200021
:1008A0001A00090030E0A00099C8A900ABC8A9004F
:1008B000BDC8A9003C28A8006028A8008428A8007A
:1008C00010002000C0418800E042880000448800F9
:1008D000C03F2000D0418800F042880010448800CA
:1008E0003D003700F0FF2F00A0418800C042880083
:1008F000E04388001000200080418800A04288006A
:10090000C043880090418800B0428800D0438800EE
:10091000800A20007041880090428800B04388001F
:10092000808920001A00090030E0A00099C8A900C1
:10093000B1C8A900C9C8A9003C28A8006028A8001F
:100940008428A800E01F2000C0418800E042880001
:1009500000448800D0418800F0428800104488009C
:100960001D0037002C23A900000E2000001988006C
:10097000100020004019880020F021002019880074
:1009800021E3A8000428A800130037000028EF0086
:1009900005E1A90011E1A90094E0A90084E0A90003
:1009A000C00120002016880000002000601688008A
:1009B0000060FE00C2A2AE00FDFF37000040FE0056
:1009C000C2A2AF00FDFF37000060FE00C2A2AE0071
:1009D000FDFF3700B6FE37000060FE0040A7A8000C
:1009E000200F200060088800A0022000100C880062
:1009F000A0022000000C88008461A90011E1A80079
:100A000094E0A800F0FF27001008880005E1A80086
:100A10008460AE00FEFF37008460A900FA06020081
:100A2000000000002228AF00D8FF37002248AE00A7
:100A3000080037002248A9002808E200020032001E
:100A40002828EF0027003700F0FF270040418800EA
:100A5000240037001048AE00060037001048A900F7
:100A60000228EC0010408000AA0A020000000000EA
:100A70008FFE37001648AE000A0037001648A9005E
:100A80000208E20002003A006000200002A8B7005D
:100A90000228ED0010408000AA0A020000000000B9
:100AA00083FE37000A48AE00070037000A48A90055
:100AB000F0FF2E002808E3000A003E00000021009D
:100AC0002828B400070037001C48AE000500370096
:100AD0001C48A900000021002808E300010036009E
:100AE0002828B5000428AF00870037004041800067
:100AF0002A28B400C6FF39000468AF000F00370091
:100B00000408A800C1822000828920005C0702003E
:100B10000000000001852000A28A20005C0702007E
:100B20000000000041872000C28B20005C0702000B
:100B3000000000000408A900B5FF3700C1822000B2
:100B4000E28C20005C07020000000000018520000C
:100B5000028E20005C070200000000004187200098
:100B6000228F20005C07020000000000E38C2000C0
:100B700087892000898A20000408A80013027800D1
:100B8000F40FB200930A9000F50FB2002313900007
:100B9000F60FB200DC050200000000000938E10099
:100BA000030032008381E8008783E800F3FF370009
:100BB0000408A90096FF37000500E00004003A0091
:100BC000860B7800960B9800A6139800000006008C
:100BD0006620B800504B88004800DE00404B88007B
:100BE0004800DD006A29B500001020000500500013
:100BF0000600B8004800DE00604B8800504B8000C3
:100C00000500B8004800DE000000EA000010B00057
:100C10000600B8004800DE00704B8800504B800092
:100C20000000EA000010B0000500B8004800DE0037
:100C30000000EA000010B0000600B8004800DE0026
:100C4000804B8800404B80000060010005003700A9
:100C50000B00370011003700170037001D00370068
:100C60002300370006007800800B7800804B80005E
:100C7000900B9800604B8000A013980000000600C5
:100C8000704B8000800B780006007800900B980075
:100C9000604B8000A013980000000600604B8000AD
:100CA000800B780006007800900B9800804B800045
:100CB000A013980000000600604B8000800B7800B5
:100CC000704B8000900B980006007800A0139800ED
:100CD00000000600804B8000800B7800604B800095
:100CE000900B980006007800A01398000000060002
:100CF000860B7800604B8000900B9800704B800052
:100D0000A013980000000600E006020000000000AA
:100D100082892000A38A200030408000B00EB100FC
:100D2000F10F20009002B10002003B0080804000E3
:100D3000010037008080500001003B008000EB0084
:100D4000011978000390E700F5FF3700C38B2000FE
:100D500030408000400EB100F10F20003003B100A0
:100D600002003B008080400001003700808050007E
:100D700001003B008000EB00011978000390E700C0
:100D8000F5FF3700E38C200030408000400FB100B9
:100D9000F10F20001005B10002003B0080804000F0
:100DA000010037008100780001003B008000EB006B
:100DB000011978000390E700F5FF370014FF3700B2
:100DC00085A0AE0000000600001880000608E300C1
:100DD0000300360006A8ED0006A8ED00030037006A
:100DE0000608B4000000D1003040880085A0A900AA
:100DF00000000600101680000010A3000CA8D6000A
:100E0000101680000000A30012A8D6005016800023
:100E100000F0A30018A8D6005016800000E0A30040
:100E20001EA8D600101680000050A30024A8D600EB
:100E300053002000A18020002807020000000000CD
:100E4000E68040008301E900FBFF3A000000060055
:100E50001100A70008003700F0FF2F0011019000DB
:100E60000201600003003A001100A000000F200002
:100E7000A000980000000600F0FF2F001101900074
:100E8000020160000001690003003A001100A100A6
:100E90001120A00000000600648140001209E90052
:100EA00001003200000006001110A000000F200019
:100EB000A000980000000600608040001000E000E4
:100EC000020032001008E900000006004100900016
:100ED000EA81400093094000010031000000060053
:100EE0008204780000012000800541002106900066
:100EF000B106900011049000F00F2000880350000C
:100F0000010B90000600A7000200370062054100B7
:100F1000010037000B057800F282400019007800CC
:100F200000E0A60003003700950AE9001A003A0025
:100F300000E0A10000D0A7000C0037000044E7004B
:100F40001AE0A1000C4040001300390000C0EB0083
:100F500000D0A2000610A6000F00370000E0A0009D
:100F6000E1019000830A78000B003700003CE700A5
:100F70001AE0A1000D405000070031000040EB00D6
:100F800000D0A2000610A6000300370000E0A00079
:100F9000F1019000830A7800800C78000B48E7008C
:100FA000000006008582E8008984E8000A85E800E0
:100FB0000B50E600D9FF370002057800D7FF370055
:100FC00000A0FE00849FBE00204880000060010059
:100FD0003C0037000B003700130037000429EF00F6
:100FE00040002000200C8800F0FE2F00E14A800025
:100FF00020168800611688008C080200000000009E
:101000003C00370040002000200C880070FF2F00BB
:10101000014B8000201688006116880092080200AB
:10102000000000003300370040002000200C880042
:10103000B0FF2F00214B8000201688006116880029
:1010400006A9EC00F00F20000609E300230036009B
:101050000408AF001B00370000002000900188004A
:101060000000EB000520200081892000A48A2000D8
:10107000829020003540BA00313178000408E10048
:10108000FCFF3A0005202000A18A2000C48B20002C
:10109000429220003540BA00313178000408E10066
:1010A000FCFF3A0005202000C18B2000E48C2000CA
:1010B000029420003540BA00313178000408E10084
:1010C000FCFF3A000629EF000629EC002000200072
:1010D000204888000428AF002023A800A38A280005
:1010E0000609D40063007800000C8800860802001E
:1010F000000000000429EC000060FE004F02BE006A
:101100000080FE0084E0A9000040060081902000DD
:10111000C295200005003700419220000296200071
:1011200002003700019420004296200033488000DE
:101130000400220004097800310078000304E10073
:101140001289D300FCFF3900010009001209D10007
:10115000000006002B0000002B0000002B00000008
:101160002B0000002B0000002B0000002B000000D3
:101170002B0000002C0000002D0000002E000000BD
:101180002F0000003000000031000000310000009E
:101190003200000033000000340000003500000081
:1011A0003600000037000000380000003800000062
:1011B000390000003A0000003B0000003C00000045
:1011C0003D0000003E0000003E0000003F00000027
:1011D0004000000041000000420000004300000009
:1011E00044000000450000004500000046000000EB
:1011F0004700000048000000490000004A000000CD
:101200004B0000004B0000004C0000004D000000AF
:101210004E0000004F000000500000005100000090
:101220005200000052000000530000005400000073
:101230005500000056000000570000005800000054
:1012400058000000590000005A0000005B00000038
:101250005C0000005D0000005E0000005F00000018
:101260005F000000600000006100000062000000FC
:1012700063000000640000006500000065000000DD
:1012800066000000670000006800000069000000C0
:101290006A0000006B0000006C0000006C000000A1
:1012A0006D0000006E0000006F0000007000000084
:1012B0007100000072000000730000007300000065
:1012C0007400000075000000760000007700000048
:1012D0007800000079000000790000007A0000002A
:1012E0007B0000007C0000007D0000007E0000000C
:1012F0007F000000800000008000000081000000EE
:1013000082000000830000008400000085000000CF
:1013100086000000860000008700000088000000B2
:10132000890000008A0000008B0000008C00000093
:101330008D0000008D0000008E0000008F00000076
:101340009000000091000000920000009300000057
:10135000930000009400000095000000960000003B
:101360009700000098000000990000009A0000001B
:101370009A0000009B0000009C0000009D000000FF
:101380009E0000009F000000A0000000A0000000E0
:10139000A1000000A2000000A3000000A4000000C3
:1013A000A5000000A6000000A7000000A7000000A4
:1013B000A8000000A9000000AA000000AB00000087
:1013C000AC000000AD000000AD000000AE00000069
:1013D000AF000000B0000000B1000000B20000004B
:1013E000B3000000B4000000B4000000B50000002D
:1013F000B6000000B7000000B8000000B90000000F
:10140000BA000000BB000000BB000000BC000000F0
:10141000BD000000BE000000BF000000C0000000D2
:10142000C1000000C1000000C2000000C3000000B5
:10143000C4000000C5000000C6000000C700000096
:10144000C8000000C8000000C9000000CA00000079
:10145000CB000000CC000000CD000000CE0000005A
:10146000CE000000CF000000D0000000D10000003E
:10147000D2000000D3000000D4000000D50000001E
:10148000D5000000D6000000D7000000D800000002
:10149000D9000000DA000000DB000000DB000000E3
:1014A000DC000000DD000000DE000000DF000000C6
:1014B000E0000000E1000000E2000000E2000000A7
:1014C000E3000000E4000000E5000000E60000008A
:1014D000E7000000E8000000E8000000E90000006C
:1014E000EA000000EB000000EC000000ED0000004E
:1014F000EE000000EF000000EF000000F000000030
:10150000F1000000F20000000000000001000000F7
:1015100002000000020000000300000004000000C0
:1015200005000000060000000700000008000000A1
:1015300009000000090000000A0000000B00000084
:101540000C0000000D0000000E0000000F00000065
:1015500010000000F10720009101880001E02F0039
:101560008008BB006027EF0061C7A8006047A800A3
:101570000700FC0051052000313B8800A10A200033
:10158000313B880061E7A800000000000000000077
:1015900061E7AF00FEFF370000000600F007200003
:1015A0009001880000E02F001000BA000000060043
:1015B0000000FE00000800007201000002000000B0
:1015C000000000000000000000000000000000001B
:1015D000000000000000000000000000000000000B
:1015E00000000000000000000000000000000000FB
:1015F00000000000000000000000000000000000EB
:1016000000000000000000000000000000000000DA
:1016100000000000000000000000000000000000CA
:1016200000000000000000000000000000000000BA
:1016300000000000000000000000000000000000AA
:10164000000000000000000000000000000000009A
:10165000000000000000000000000000000000008A
:10166000000000000000000000000000000000007A
:10167000000000000000000000000000000000006A
:10168000000000000000000000000000000000005A
:10169000000000000000000000000000000000004A
:1016A000000000000000000000000000000000003A
:1016B000000000000000000000000000000000002A
:1016C000000000000000000000000000000000001A
:1016D000000000000000000000000000000000000A
:1016E00000000000000000000000000000000000FA
:1016F00000000000000000000000000000000000EA
:1017000000000000000000000000000000000000D9
:1017100000000000000000000000000000000000C9
:1017200000000000000000000000000000000000B9
:1017300000000000000000000000000000000000A9
:101740000000000000000000000000000000000099
:101750000000000000000000000000000000000089
:101760000000000000000000000000000000000079
:101770000000000000000000000000000000000069
:101780000000000000000000000000000000000059
:101790000000000000000000000000000000000049
:1017A0000000000000000000000000000000000039
:1017B00000000000FFFFFF00FFFFFF00FFFFFF0032
:1017C000FFFFFF00FFFFFF00FFFFFF00FFFFFF0025
:1017D000FFFFFF00FFFFFF00FFFFFF00FFFFFF0015
:1017E000FFFFFF00FFFFFF00FFFFFF00FFFFFF0005
:1017F000FFFFFF00FFFFFF00FFFFFF00FFFFFF00F5
:0200000401F009
:100000000F000000000000000300000001000000DD
:10001000FB000000C20000007A000000C3040000E2
:04002000B500000027
:00000001FF
